:020000040800F2
:10000000000400109D0B00082F260008352600086C
:100010003B26000841260008472600080000000093
:10002000000000000000000000000000532600084F
:100030004D26000800000000592600085F26000831
:100040006526000865260008652600086526000864
:100050006526000865260008652600086526000854
:100060006526000865260008652600086526000844
:100070006526000865260008652600086526000834
:100080006526000865260008652600086526000824
:100090006526000865260008652600086526000814
:1000A0006526000865260008652600086526000804
:1000B00065260008652600086526000865260008F4
:1000C00065260008652600086526000865260008E4
:1000D00065260008590A0008650A0008710A000828
:1000E00065260008652600086526000865260008C4
:1000F00065260008652600086526000865260008B4
:1001000065260008652600086526000865260008A3
:100110007D0A0008890A000865260008652600088F
:100120006526000865260008652600086526000883
:100130006526000865260008652600086526000873
:100140006526000865260008652600086526000863
:100150006526000865260008652600086526000853
:100160006526000865260008652600086526000843
:100170006526000865260008652600086526000833
:100180006526000865260008F0B50546541C047075
:1001900005F8013F83F47F4383F0FF03114FDBB287
:1001A000023237F8133092B283F0FF038E46C1F16A
:1001B00002047444A4B294424FEA13260AD21EF8F1
:1001C000014B05F8014F6340DBB2B6B237F813308C
:1001D0007340ECE7022A38BF02228354013292B204
:1001E0008654F0BD282A000838B590F8333004460C
:1001F000052B00F28380DFE803F0030E253A4884E4
:10020000C36A1970838C89B28B42018476D3012032
:1002100084F8330038BDC36A3C4A597081F47F4189
:1002200081F0FF01038CC9B2013B32F811209BB26F
:10023000038482F0FF020220E083E286ABB184F8FF
:10024000330020E0C38BC26A581CE083D154E28E95
:100250002E4B5140C9B233F8113083EA1223E386A2
:10026000238CE28B02339A420DD1032309E0C28E24
:10027000264B5140C9B233F8113083EA1223C386AA
:10028000042384F83330012038BD052380F833304F
:10029000C38E1E4A5940C9B232F81120B2EB132F57
:1002A00028D1C06A4578290609D5237F5D406A06B2
:1002B00029D163F07F0323770123A38623E035B997
:1002C0002046294601F0BEFE84F822501BE094F837
:1002D0002210A94201D1204609E0236884F8225067
:1002E00013B10230218C9847E36A5978204601F017
:1002F000A9FE08E0836B0133836302E0052384F8E1
:100300003330002038BD022038BD00BF282A000845
:1003100020B1036803481B1A5842584100F00100FD
:10032000704700BF55AA55AA2DE9F04F85B00E467B
:1003300090460193BDF838B0BDF84090009000B9E8
:10034000FEE701B9FEE7BBF1000F02D0019B03B944
:10035000FEE7B9F1000F02D00F9B03B9FEE71BF1D6
:100360000003B26918BF012319F1000A18BF4FF04A
:10037000010A1AB9BAF1000F00D0FEE772690AB992
:1003800003B1FEE72C4A03931778022F4ED8791C4D
:10039000DFF8B4C01170282202FB07F50CEB05044E
:1003A00020460021CDF808C001F0D2FDDDF808C0DC
:1003B000039B224AA6604CF80520C4F804802373EE
:1003C00084F80DA06646DBB1103565445A462846D0
:1003D000019902F0B4F8A36819495B6940462246C6
:1003E0009847A368D3F810B0BBF1000F08D063683A
:1003F0000193284601F0F5FF019B01461846D847B6
:10040000BAF1000F0ED028235F43F01937441C3097
:100410000F994A4602F093F8BB680A499B69404627
:1004200022469847009B00201C6001E04FF0FF30FF
:1004300005B0BDE8F08F00BFFA01002055AA55AA0B
:10044000F7210008B321000858000020102808B543
:1004500000D9FEE7034B53F8200000F051FF80B2B3
:1004600008BD00BFA8280008102800D9FEE7024BED
:1004700053F8200000F034BFA8280008034A906811
:10048000D36851690344194402F072B8803F0008F0
:1004900008B502F08AF800F07BFC054BD968986833
:1004A000890800F07DFCBDE8084000F087BC00BF73
:1004B000803F000800B599B001A800F05FFD0B492E
:1004C000019A0B4BB2FBF3F30B600A4B1A600A4A1A
:1004D000D36843F08073D360084A1368002043F068
:1004E0000103136019B05DF804FB00BFD4000020C5
:1004F00040420F00D0000020F0ED00E0001000E0CE
:1005000009490A4B0A6830B51D6800230C68A21A15
:100510001344B3FBF5F2824204D2801A05FB123376
:100520002246F3E7002030BD041000E0D400002094
:10053000034B1868034B1B68B0FBF3F0704700BF18
:10054000041000E0D40000202DE9F04782460D465B
:1005500001B9FEE7CAF800104FF000082B795FFAE6
:1005600088F7BB4249D918247C432E68244A335962
:10057000934206EB04091AD007D8B3F1904F10D07C
:10058000A2F5806293420FD029E01E4A934214D014
:1005900002F58062934213D0A2F50062934209D023
:1005A0001DE04FF400300DE04FF480200AE04FF4DE
:1005B000002007E04FF4801004E04FF4001001E049
:1005C0004FF48000012100F04FFED9F810203AB11D
:1005D0003059B9F80410D2B202F0A1F800E0FEE7F9
:1005E000305909F1040102F050F8DAF800003946F8
:1005F00002F006F808F10108B0E70020BDE8F08736
:100600000008004800100048074B1A681AB9EFF3B9
:10061000108206490A604FF0010080F310881A68C2
:1006200001321A6000207047DC000020D800002052
:1006300007B500F0FBFA00F077FB00211F4800F03F
:1006400081FC4FF4407000F03DFC042000F084FC7D
:10065000FFF730FF1A48012100F006FE194801217A
:1006600000F01AFE0121184800F00AFE684602F068
:1006700048F801238DF80730694641F6FF734FF0C3
:100680009040009302F001F84FF6FF7369460F485F
:10069000009301F0FAFF69460D4801F0F6FF694644
:1006A0000C4801F0F2FF69460B4801F0EEFF0B48E1
:1006B000694601F0EAFF03B05DF804FB00000008A2
:1006C00057007E3137C8FE32017807000004004829
:1006D00000080048000C00480010004800140048C2
:1006E00008B5FFF791FF002001F03AF8012001F072
:1006F00037F8BFF34F8F0549054BCA6802F4E06233
:100700001343CB60BFF34F8FFEE700BF00ED00E067
:100710000400FA050268054B9A4200D0FEE74368E0
:1007200003491868012202F03AB800BF443322118D
:10073000050105000268054B9A4200D0FEE74368B8
:1007400003491868012202F02AB800BF443322117D
:100750000701070030B50268254B9A4285B0044670
:1007600000D0FEE743681A68D3699BB2ADF80E303B
:10077000938CDBB28DF80A30BDF80E200023910671
:100780008DF80B3011D5056A9DF80A208DF80D20E3
:100790005DB10DF10B020092406A0DF10D010122D5
:1007A000A84710B9636B01336363BDF80E200023C3
:1007B00012068DF80C3019D5A56A8DB103AA0092E6
:1007C000E06A01220DF10D01A8476368024620B1DD
:1007D0001B689DF80D201A8508E01868054903E09C
:1007E0006368044918682A4601F0D9FF05B030BD96
:1007F000443322110701070070B583695A0786B098
:10080000044613D54368986880B15A681AB1197DB7
:10081000D2B201F084FF616888680C3101F035FFC5
:10082000636819491868012201F0B9FFA3691B0721
:100830000ED56368986958B15A6822B193F82410AC
:10084000D2B201F06CFF616888691C3101F01DFFB4
:1008500004F108060FCE6D460FC596E8030085E843
:10086000030023B1019B13B94FF4805301936368D4
:100870006946186800F064FD63680121186801F09A
:100880006BFF06B070BD00BF0501050030B50568FF
:10089000064CA54200D0FEE7C2628269816242F046
:1008A00008028261BDE83040FFF7A6BF4433221141
:1008B00030B50568064CA54200D0FEE74262826969
:1008C000016242F004028261BDE83040FFF794BF4C
:1008D0004433221170B50668194D049CAE4200D015
:1008E000FEE790F8305055BB012905D0022904D10C
:1008F0004FF48051C16000E0C560032B05D0042B8C
:1009000006D0022B07D1002304E04FF4405301E04E
:100910004FF400530361022A05D0032A06D0012AAE
:1009200007D1002304E04FF4806301E04FF4C0637B
:10093000436104B18460BDE87040FFF75DBF70BDE6
:100940004433221110B5074A0468944200D0FEE7F0
:1009500090F8302022B98160BDE81040FFF74CBF0D
:1009600010BD00BF443322112DE9F341394B144629
:1009700002689A42054600D0FEE743681868066898
:10098000013906F0010607295FD8DFE801F0143DC0
:10099000454D4F044D54237895F838200024009499
:1009A00068468DF8013001238DF800208DF8033062
:1009B00000F092FA47E00268247822F00102026017
:1009C0009A68B2B10C3393E8030014F001088DE883
:1009D000030014BF02230123104669468DF8073037
:1009E00001F053FE6B684FF480311868424601F005
:1009F000BCFE6B689A690AB318684FF40031C4F3FF
:100A0000400201F0B2FE19E00368217823F00103EF
:100A1000036001F0B2FE11E00368217823F00103C6
:100A2000036001F0B3FE09E0083300E018330FCB98
:100A300084E80F0002E0237885F830306B681A688C
:100A400013681E431660002001E04FF0FF3002B033
:100A5000BDE8F08144332211014B1868FFF77ABEDC
:100A600060010020014B1868FFF774BE640100208C
:100A7000014B1868FFF76EBE68010020014B186833
:100A8000FFF768BE58010020014B1868FFF762BEEF
:100A90005C0100202DE9F74F0B68364A93428246ED
:100AA0008B461ED00CD8A2F50062934214D002F5FA
:100AB0008062934258D1304C4FF02708256819E0E6
:100AC0002E4A934212D002F5684293424CD12C4CEC
:100AD0004FF0250825680DE02A4C4FF026082568C0
:100AE00008E0294C4FF03408256803E0274C2568BE
:100AF0004FF035081DB1CAF80050002036E0244BF5
:100B00001E78012E30D8721CDFF88C901A703C22AF
:100B1000564309EB06072946384601F019FA06F153
:100B200008001C4BC7F804B0484487F8388049F8DF
:100B3000063001F006FEBD61CAF8007097F8383043
:100B400001958DF8043008238DF8053001A80123A4
:100B500027608DF8073000F0BFF97B684FF48051B3
:100B6000186801F033FEC8E74FF0FF3003B0BDE86E
:100B7000F08F00BF004C0040680100200050004092
:100B80006001002064010020580100205C01002069
:100B9000FB01002044332211E0000020194CA24642
:100BA000194A1A48536A43F4E0235362184B5968B0
:100BB00041F040415960D96841F00071D960D9686D
:100BC00041F08071D960D2F88830124943F4700343
:100BD000C2F88830104A121A01F020F90F48104A62
:100BE0000021121A01F0B4F90E480F4A0021121A1E
:100BF00001F0AEF9A5214FF47072204601F0A8F97A
:100C000000F042FC0000001000ED00E000000020B9
:100C100030EF00E0302C0008580000205800002081
:100C2000340900200004001000040010394AD2F8F2
:100C3000883043F47003C2F88830374B1A6842F0AA
:100C400001021A605968354A0A405A601A6822F04F
:100C5000847222F480321A601A6822F480221A60A8
:100C60005A6822F4FE025A60DA6A22F00F02DA624F
:100C7000196B2B4A82B00A401A6300229A600092D4
:100C800001921A6842F480321A601A6802F4003243
:100C90000192009A01320092019A1AB9009AB2F5B3
:100CA000A04FF2D11A6812F4003218BF012201924B
:100CB000019A012A05D0174B4FF000629A6002B0EA
:100CC0007047184A122111605A685A605A685A606F
:100CD0005A6842F480625A605A6822F47C125A6060
:100CE0005A6842F4E8125A601A6842F080721A6038
:100CF0001968094A8901FBD5516821F00301516047
:100D0000516841F0020151605A6802F00C02082A51
:100D1000FAD1D0E700ED00E0001002400CC07FF8EF
:100D2000CCFC00FF00200240144A1549536803F030
:100D30000C03042B10B501D0082B01D0114B12E08D
:100D400053685068C00349BFD06A0F480D4C00F08B
:100D50000F00C3F3834348BF013003F1020348BFD0
:100D6000B4FBF0F043430B605368084AC3F303132A
:100D7000D25C0B68D3400B6010BD00BF0010024076
:100D80000000002000127A0000093D00340000201D
:100D9000024A936843F001039360704700300240B9
:100DA00000EB81018842044B03D050F8042B1A60F9
:100DB000F8E71868704700BF00300240014B186820
:100DC000704700BF00300240044B1A6810B142F077
:100DD000100201E022F010021A6070470020024069
:100DE000044B1A69120641BF034A5A6002F1883265
:100DF0005A6070470020024023016745024A136988
:100E000043F080031361704700200240084BDA680A
:100E1000D10709D4DA68D20608D4DB6813F0040FCE
:100E200014BF032004207047012070470220704740
:100E30000020024038B505464FF4302001F014FC84
:100E4000042811D1094C236943F002032361656131
:100E5000236943F0400323614FF4302001F004FC88
:100E6000236923F00203236138BD00BF0020024044
:100E700073B5002306464FF430200D46019301F070
:100E8000F3FB042819D10E4C236943F001032361BD
:100E9000ABB233804FF4302001F0E6FB042808D1D8
:100EA00002360196019B2D0C1D804FF4302001F07D
:100EB000DBFB236923F00103236102B070BD00BF97
:100EC0000020024040F0BF60024B40F40030D86088
:100ED000704700BF00ED00E0C278037810B50AB398
:100EE000164AD4684278E443C4F30224C4F10401EE
:100EF00002FA01F10F22E240847822400A4303F112
:100F0000604303F561431201D2B283F800230378F2
:100F10000122590903F01F0302FA03F3084A42F8B9
:100F2000213010BD5A09012103F01F03994002F13D
:100F30002003034A42F8231010BD00BF00ED00E07B
:100F400000E100E021F0604121F07F01014B084306
:100F50009860704700ED00E0044B1A6804280CBF4D
:100F600042F0040222F004021A60704710E000E030
:100F7000014B1860704700BF20000E422DE9F04180
:100F80009B4F7B6803F00C03042B05D0082B06D085
:100F9000984A0260B3B916E0964B036012E07B6892
:100FA0007968C3F383439A1CCB0349BFFB6A924B16
:100FB000904903F00F0344BF0133B1FBF3F35343F4
:100FC000036000E000237A688C4EDFF834C2C2F37D
:100FD0000312B45C0268E4B222FA04F141607D6855
:100FE000C5F30225755D21FA05FEC0F808E07D68AD
:100FF000C5F3C225755DEDB2E940C160FE6AC6F376
:10100000041808F00F0618F0100F3CF81660E046C0
:10101000B6B204D01EB1B3FBF6F6066100E0026181
:10102000FE6AC6F3442C0CF00F061CF0100F38F8C3
:101030001660B6B204D01EB1B3FBF6F6466100E00E
:1010400042613E6BF6065ABF6A4E866182613E6B14
:10105000B6065ABF674EC661C2613E6B76065ABF7E
:10106000644E066202623E6BF60506D59A4204D1D2
:10107000A54202D15600466200E041623E6BF60492
:1010800006D59A4204D1A54202D15600866200E0FC
:1010900081623E6BB60506D59A4204D1A54202D1C3
:1010A0005600C66200E0C1623E6B760506D59A42E4
:1010B00004D1A54202D15600C66400E0C1643E6B73
:1010C000360506D59A4204D1A54202D156000665DE
:1010D00000E001653E6BB60406D59A4204D1A542F4
:1010E00002D15600466500E001653E6B360406D528
:1010F0009A4204D1A54202D15300836500E0816584
:101100003C6B3B4BA40701D1816315E0196B01F0E7
:101110000301012901D182630EE0196B01F0030183
:10112000022902D14FF4004305E01B6B03F00303D7
:10113000032B01D12F4B8363396B2D4B11F4403FAF
:1011400002D1C0F83CE018E0196B01F44031B1F570
:10115000803F01D1C26310E0196B01F44031B1F559
:10116000003F02D14FF4004306E01B6B03F4403311
:10117000B3F5403F01D11F4BC363396B1C4B11F4D6
:10118000402F02D1C0F840E018E0196B01F4402173
:10119000B1F5802F01D1026410E0196B01F44021F8
:1011A000B1F5002F02D14FF4004306E01B6B03F4AE
:1011B0004023B3F5402F01D10E4B0364396B0C4B28
:1011C00011F4401F02D1C0F844E023E0196B01F490
:1011D0004011B1F5801F01D142641BE0196B01F48D
:1011E0004011B1F5001F0DD14FF4004311E000BFD5
:1011F0000010024000127A0000093D004400002067
:10120000140000201B6B03F44013B3F5401F01D101
:10121000134B4364396B134B11F4400F03D1C0F8E7
:1012200048E0BDE8F081196B01F44001B1F5800F91
:1012300002D18264BDE8F0811A6B02F44002B2F57B
:10124000000F02D14FF4004306E01B6B03F4400390
:10125000B3F5400F01D1024B8364BDE8F08100BFBC
:1012600000127A0000100240044B5A6909B1104381
:1012700001E022EA00005861704700BF0010024000
:10128000044B9A6909B1104301E022EA0000986119
:10129000704700BF00100240044BDA6909B11043E7
:1012A00001E022EA0000D861704700BF0010024050
:1012B000044BDA6809B1104301E022EA0000D8606B
:1012C000704700BF00100240044B1A6909B1104377
:1012D00001E022EA00001861704700BF00100240E0
:1012E00082B000230193054B0193019B03EB800027
:1012F0000190019B196002B0704700BF5028004068
:1013000082B000230193054B0193019B03EB800006
:101310000190019B186802B0704700BF5028004040
:101320000549064ACB68024042F0800203F0800380
:1013300063EA0203CB607047002800407FFF010092
:10134000036823F0010330B50360436823F440527F
:101350008B680D46134343606A68C968036811438C
:101360002A6923F4B0530A4323F00C0313430360A8
:10137000836823F440726B6999B013438360044619
:1013800001A8FFF7FBFD184B9C4201D10F9B0EE01B
:10139000164B9C4201D1109B09E0154B9C4201D198
:1013A000119B04E0134B9C420CBF129B139B2268C1
:1013B000296812F4004F18BF5B00B3FBF1F201FB88
:1013C0001233B3EB510F236828BF01321B0441BF16
:1013D0004FF6F073C2F34201134041EA030292B2A6
:1013E000A28119B030BD00BF003801400044004068
:1013F00000480040004C0040044A13680133136069
:10140000034B0146186800F0A0BF00BF7C0100201C
:101410005005002007B50E4A1368013313600D4BC9
:10142000012218680DF10701002300F099FF01283F
:1014300003BF094A9DF8070013684FF6FF7008BF05
:10144000013300B208BF136003B05DF804FB00BFB6
:10145000740100205005002070010020074B0A464F
:10146000012110B5197006490B68044601330B6061
:1014700004482146BDE8104001F026B83B03002097
:10148000C4010020C80100202DE9F84FFFF7D0F873
:1014900000F016F901F0C0F901F0C5F9044650B9A1
:1014A0004FF4FA7001F085F86D4B1C706D4B0722FC
:1014B0001A7001F0CCF94FF480726B486B4901F05F
:1014C0003EF86B486B4900F0ECFDFFF731F807463A
:1014D000384601F079F88146654800F02FFE6448EF
:1014E00000F0FDFD644B188008B10328F4D15E487C
:1014F00000F06CFF3E280FD900245B4800F07DFF10
:101500005E4A105501343F2CF7D15D490B681046F7
:1015100001330B6000F06EF9524EDFF888813378AA
:10152000584D594CDFF880A1092B2CD8DFE803F087
:10153000050B2B2B2B05161F2B0541F28833C8F802
:10154000003064230FE041F28833C8F80030642390
:101550002B6040F6C413236032231BE040F6C41313
:10156000C8F8003032232B600023236014E04FF0D2
:10157000000B64235846C8F800B02B6000F0E8F870
:10158000C4F800B008E041F288326423C8F80020B3
:101590002B602260CAF80030B8F80000296820B13A
:1015A00089B24A4601F01AF901E000F0D9F8208822
:1015B000DAF8001020B189B24A4601F00FF901E0D3
:1015C00000F0C6F8314B324C9945227806D9337871
:1015D000072B05D0B3FA83F35B0902E0002300E098
:1015E0000123134303F001030020237000F0AEFB3E
:1015F0002378002B3FF46CAF264B1B78002B7FF435
:1016000067AF254B9C6823685B0C5B04B3F1005FFC
:1016100002D0B3F1805F1FD1FFF7F0FB4FF0FF3036
:101620000121FFF745FE4FF0FF300121FFF74CFE8F
:101630004FF0FF300021FFF73BFE4FF0FF3000215D
:10164000FFF742FE154A63681360154A136022686B
:1016500082F3088898473BE70C23337038E700BFD4
:101660005400002043050020C80100203B02002058
:101670008001002018290008F8010020FC0100204A
:101680006C0100200800002004000020808D5B0019
:101690003F0400203B030020803F00087801002029
:1016A0004C050020100000200C00002008B5034667
:1016B0000A460248194600F052FD08BD800100208C
:1016C00010B5012086B0FFF77FFB114800F038F815
:1016D00005A81049FFF7DEF900B1FEE70E4C0F4AEE
:1016E00001924FF480730093029320460C49059AAF
:1016F0000C4BFEF719FE00B1FEE701214FF46143E8
:10170000009320680A46022300F0CAFD06B010BD0F
:101710006C29000874290008500500205406002098
:10172000E828000854050020032800D9FEE7034BF1
:1017300089B233F81000FEF797BE00BF282C0008CE
:10174000014600B9FEE70148FEF7FEBED4010020C5
:10175000024BC1B2186800F03DBF00BFD4010020A9
:10176000024BC1B2186800F04BBF00BFD40100208B
:1017700030B1012807D1054B98685B681844704761
:10178000024B586870470020704700BF5807002080
:10179000034B1B780BB9FEF77BBE0020704700BFE0
:1017A000F30800202DE9F0410F4CD4F80880E768D9
:1017B0006569A679FFF7ECFF63792279E17943EA5D
:1017C00002220A4B01241C70094B0024EDB21C704C
:1017D00003245C70C3F804809F601D735E73DA811C
:1017E00019745861BDE8F081803F0008460500206B
:1017F000700700202DE9F04F054610F8013BDFF897
:10180000F4C2A849A84FDFF8F0A23B7089B0DA090A
:1018100001929DF804208CF80020C3F380120A7016
:10182000C3F340120092A14A04939DF80030CDF812
:101830001CC00591137001F019F86B1DCAF8000067
:1018400004461846029301F011F8DFF8B0920390B5
:10185000C9F800009648AA7902709648EE79067099
:1018600095482E7ADFF8988295F805B0067005F154
:101870000900069288F800B000F0F8FF8F4E306043
:1018800005F10D0000F0F2FF706005F1110000F0AD
:10189000EDFF049B0199DDF81CC0B06003F01F034D
:1018A0003B70CDF810C0069A49B18548294605F12C
:1018B000400E51F804CB40F804CB7145F9D1013BFF
:1018C0000A2B00F20D82DFE813F01F010B020B0060
:1018D00069018401870148008D01B3010B02DF011A
:1018E000784D2B78072B04D1774B1B785B4504D8B8
:1018F000F6E113B10C2B40F0F381BBF1000F01D0E6
:10190000FFF750FF002398F800102B7018234B436B
:101910006E4A6F4E12F803E0D4186E4B6E4A83F88D
:1019200000E0637803F0010111706C4AC3F34003D7
:1019300013700FCC0FC694E8030086E80300BEF1D5
:10194000000F02D0BEF1010F02E000F029FE0128D5
:1019500000F0C68108232B7044E05A4B1978012906
:101960001E4600F2BD810099DFF8988100293ED023
:10197000D8F80030002B40F08F80594B019283F84B
:1019800000B0584BC8F80010E81D1C6000F06EFF56
:10199000554B019A1860554B1A706FF0370303EBE3
:1019A0008202382303FB0424BBF1000F03D0BBF1F8
:1019B000010F05D008E0464B9B689C4206D903E026
:1019C000434B1B7B9C420FD90A2366E0414B1B789B
:1019D00013B1012B04D007E0FEF750FD012803D01E
:1019E000082333703A785AE00123337078E1D8F84D
:1019F0000010002950D03B4A1268944201D90322BA
:101A000046E001398C4242D1013A94420ABF374B39
:101A10000E231B7800932F4B1C786CBB029D204635
:101A2000009BE2B29A4225D2284600F01FFF2C4AC2
:101A3000C9F800001078FFF79BFEDAF800204FF09D
:101A4000380B0BFB02FB0BEB840B834403220020BF
:101A500050B95846D9F800100192FFF709FA031F50
:101A600058425841019A00E00120013AF0D1013476
:101A70000435D5E7012804D0082333701C4B3A788D
:101A80001A60D8F800300133C8F8003028E102228B
:101A90001A70174B1C6023E1082333700722144B84
:101AA0001A601DE14405002045050020490500207D
:101AB000AE080020B2080020B10800206008002015
:101AC0006E08002043050020460500207007002016
:101AD00058070020F30800206D0800206C08002043
:101AE000AF080020EC010020F00100204705002095
:101AF000E801002048050020DC01002054070020F8
:101B0000B0080020E4010020FFF74CFE7E4B0122CC
:101B10001A7002225A7098F800201946CAB99A70B1
:101B2000DA701A715A719A71784B1C78CC7113461D
:101B3000A2420ADA764D182000FB02505500407888
:101B4000A84003439BB20132F2E71A0A0A724B72B1
:101B50001FE06F499A71501E182404FB00114A7B44
:101B6000DA710A7B88681A72CA8949695871050E48
:101B70000C0E9D709C72050C0C0CDD70DC72050A5D
:101B80000C0AD0B2120A1D7158721C7359739A73E1
:101B9000D8733F215F48FFF789FDA1E0039A45F61E
:101BA000FE239A4203D14FF6FF7000F05BFE002047
:101BB0003168FFF7B9FD01207168FFF7B5FD02201C
:101BC000B168FFF7B1FDFFF719F9534B01221A7005
:101BD00086E0FEF785FD83E0504A00231360504AFB
:101BE00013707DE04E4C2378012B79D14B4D4D4A3B
:101BF0002B681168013B8B4216460ED100232B60E7
:101C0000494B1B780BB1052306E0484B1F68FFF7D3
:101C1000BFFD8742F7D00B2323702B683268013B4E
:101C200093425DD23D4B00221A600423237057E09B
:101C30003B4B1878194618BB3D4B83F800B03D4B21
:101C40001C603D4B1A600E3A0E2303FB0424BBF1CB
:101C5000000F05D0BBF1010F09D1384B1A7B01E011
:101C6000364B9A68944294BF0024012414B10A238D
:101C70000B7007E0324B00221A6006230B702FE036
:101C800008221A7009220AE71F4B2E4901221A70F6
:101C90000C225A70224A10789871022815460CBFFF
:101CA0000A6809681B4801BF110E9970110CD970A0
:101CB00017BFC1F30724110A0022DC7019714FF01D
:101CC00000045A714FF03F0118BF9A70DC711C720A
:101CD0005C72FFF7EBFC2B78052B04BF104B1C70DC
:101CE000049B1B78012B0CD11748059B1A7843786D
:101CF000134300F8013F3F2109B0BDE8F04FFFF763
:101D0000D5BC09B0BDE8F08FF408002046050020DE
:101D100070070020F50800203F040020E4010020A7
:101D200043050020EC010020AF080020F001002056
:101D30004A050020F4010020E0010020580700209F
:101D4000D8010020E80100206E0800202DE9F84F9E
:101D5000294F3B78062B4DD1284B294D294801228C
:101D60001A700A225A702A685A71110E9970110C51
:101D7000D970110A1971016801398A421C4604BFE1
:101D8000214B93F800A0804618BF4FF00E0A4FF089
:101D900000095FFA89F3534518D22B684FEA890688
:101DA0004FF0380B0BFB036B184B1878FFF7E0FC78
:101DB000174B06360BEB00011A78A01900F061FDF5
:101DC00008B908233B7009F10109E2E72B68D8F84C
:101DD000002010480133013A93422B6081BF052354
:101DE0003B700D4B0A2288BF1A603F21BDE8F84FB7
:101DF000FFF75CBCBDE8F88F43050020B308002066
:101E0000D8010020F4010020E00100204A05002054
:101E1000F3080020B4080020E8010020844641EACD
:101E2000000313F003036DD1403A41D351F8043B52
:101E300040F8043B51F8043B40F8043B51F8043BA4
:101E400040F8043B51F8043B40F8043B51F8043B94
:101E500040F8043B51F8043B40F8043B51F8043B84
:101E600040F8043B51F8043B40F8043B51F8043B74
:101E700040F8043B51F8043B40F8043B51F8043B64
:101E800040F8043B51F8043B40F8043B51F8043B54
:101E900040F8043B51F8043B40F8043B51F8043B44
:101EA00040F8043B51F8043B40F8043B403ABDD2B3
:101EB000303211D351F8043B40F8043B51F8043B55
:101EC00040F8043B51F8043B40F8043B51F8043B14
:101ED00040F8043B103AEDD20C3205D351F8043BE4
:101EE00040F8043B043AF9D2043208D0D2071CBFB0
:101EF00011F8013B00F8013B01D30B8803806046D9
:101F0000704700BF082A13D38B078DD010F003034E
:101F10008AD0C3F10403D21ADB071CBF11F8013BBE
:101F200000F8013B80D331F8023B20F8023B7BE70D
:101F3000043AD9D3013A11F8013B00F8013BF9D238
:101F40000B7803704B7843708B78837060467047D2
:101F500070B4840746D0541E002A41D0CDB2034647
:101F600002E0621EE4B3144603F8015B9A07F8D15D
:101F7000032C2ED9CDB245EA05250F2C45EA05459F
:101F800019D903F110022646103E0F2E42F8105CBC
:101F900042F80C5C42F8085C42F8045C02F1100262
:101FA000F2D8A4F1100222F00F0204F00F04103254
:101FB000032C13440DD91E462246043A032A46F840
:101FC000045BFAD8221F22F003020432134404F007
:101FD00003042CB1C9B21C4403F8011BA342FBD17A
:101FE00070BC704714460346C2E700BF10B5C36813
:101FF0000446984763691844A06110BDF8B5836A28
:1020000004461D788368E12098470335EDB2002728
:10201000FBB2AB4212D2A36ADE5DA368E12E04D10B
:10202000E0209847A368012005E0E02E304602D169
:102030009847A368304698470137E9E7237C013386
:102040002374F8BD10B541F08003002104460A4610
:10205000806AFEF799F82046BDE81040FFF7CEBF32
:1020600010B590F8324002466CB1012C17D1E1292D
:1020700003D1002382F8333011E0E0290BD1002393
:1020800080F832300BE00124E12980F83240F0D0B2
:10209000A14208BFE121BDE81040FEF7A5B801202C
:1020A00010BD4B6903608B694360CB6983600B6A29
:1020B000C360CB8943740B6943618B89C3848B886C
:1020C00083848B6883620B68C36200230374038676
:1020D000FF2380F822300377022383867047838EA4
:1020E00010B5044683B9C3689847A369984209D9D3
:1020F000227C637C9A4217D22046FFF77FFF20465E
:10210000FFF774FF012017E0012B08BFB0F8403043
:102110004FF0020203BF1343A0F840308286A2862C
:102120000CBF0320002007E0B4F84030022023F069
:102130000203A4F84030A08600B210BD38B50546B1
:1021400000246B689847431C014606D02846C9B254
:10215000FFF786FF02280446F3D120B238BD10B540
:102160000446501CE38C98421FDAA38E022B1ED12A
:10217000237F03F07F030133180648BF0123237731
:10218000B4F84030A06A23F00203A4F840300023E2
:10219000A3862374237FFDF7F7FF2046FFF72EFF6A
:1021A0002046FFF723FF012010BD042010BD0520AD
:1021B00010BDF8B504460F4615461E46FEF7A8F8B2
:1021C00000B9FEE707B9FEE705B9FEE7637B03B98F
:1021D000FEE71C342A462046394600F024F905461D
:1021E00010B1069B00221A701EB1204600F0EEF8D6
:1021F00030802846F8BDF8B504460F4615461E4601
:10220000FEF786F800B9FEE7237B03B9FEE710343A
:10221000012D204603D1397800F040F903E039461A
:102220002A4600F051F9054610B1069B00221A70AB
:102230001EB1204600F0D5F830802846F8BDF8B52C
:102240000F461446054600B9FEE7437B03B9FEE797
:1022500083685B6A00F11C063BB1406898478307BE
:1022600003D4304600F0C5F815E0304600F0B9F868
:10227000844212D822463046394600F025F90446F9
:1022800048B1AB68DF6837B130466D6800F09EF842
:1022900001462846B8472046F8BD6FF00100F8BD5A
:1022A0002DE9F3410546884617461E46FEF730F8ED
:1022B00058B1AB685C685CB1089B009368684146A4
:1022C0003A463346A047002003E04FF0FF3000E0DD
:1022D000204602B0BDE8F0812DE9F84F05460F46D3
:1022E0001446FEF715F860B36B7B03B9FEE705F102
:1022F0001C08404600F065F826468246F6B1564571
:10230000324628BF52462846394692B2FFF797FF19
:10231000002802DB361A0744F0E7831C13D1AB68B0
:10232000D3F80C90B9F1000FE8D04046D5F804B0CE
:1023300000F04CF801465846C847DFE72046BDE8A4
:10234000F88F4FF0FF30BDE8F88F07B502AB0122E0
:1023500003F8011D1946FFF7BFFF03B05DF804FB4A
:102360002DE9F84F044690461D460F4601B9FEE799
:1023700002B9FEE7FDF7CCFF00B9FEE7237B9BB96E
:10238000FEE7A368D3F81090B9F1000F07D05046CC
:10239000D4F804B000F025F801465846C8476DB19E
:1023A000012000F006F9013D04F1100A50463946BB
:1023B000424600F038F806460028E2D03046BDE834
:1023C000F88F008908B1013880B270478188C288CF
:1023D000008993B289B28B4238BF1B18581A80B259
:1023E000704710B50489FFF7F1FF013C201A80B255
:1023F00010BDC3889BB283807047F8B58488068976
:1024000007680546A4B2FFF7E1FF40B1631C385DE1
:102410009BB2B34228BF0023AB8080B201E04FF6ED
:10242000FF7000B2F8BD2DE9F84F14468588078982
:10243000D0F8008083468946FFF7C8FFA04228BF36
:10244000204684B2ADB234B34FF0000A7E1BB6B260
:10245000A64228BF2646012E04D118F8053009F8F7
:102460000A3006E009EB0A0008EB05013246FFF7E7
:10247000D5FCA41B354406EB0A00ADB2A4B21FFA8A
:1024800080FABD4228BF0025002CDFD1ABF80450F4
:102490005046BDE8F88F2046BDE8F88F2DE9F041A1
:1024A000C4880689076805468846A4B2FFF799FFE5
:1024B00040B1631C9BB2B34228BF002307F80480DD
:1024C0000120EB80BDE8F0812DE9F84F1446C58866
:1024D0000789D0F8008083468946FFF782FFA04233
:1024E00028BF204684B2ADB234B34FF0000A7E1B41
:1024F000B6B2A64228BF2646012E04D119F80A30EA
:1025000008F8053006E008EB050009EB0A01324641
:10251000FFF784FCA41B354406EB0A00ADB2A4B25D
:102520001FFA80FABD4228BF0025002CDFD1ABF88E
:1025300006505046BDE8F88F2046BDE8F88F0023CE
:1025400083800160C3800281704708B5402001216B
:10255000FEF78AFE4FF080500121FEF79DFE4FF4FA
:102560000050BDE80840FEF7DBBE0120FEF700BDCD
:10257000F8B505460F460024BD420DD25CB90326CE
:102580002846FEF757FC042802D0013EF8D101246A
:1025900005F50065F0E7012484F00100F8BD7047FF
:1025A00008B5FEF71DFC012008BD40200121FEF703
:1025B0005BBE10B504462CB14FF47A70FDF7A0FF56
:1025C000013CF8E7204610BD10B50446FDF7B0FF0A
:1025D000001B10BD00B9FEE703798B420FD901EB58
:1025E00041010268CB00D118087D496818B1D05864
:1025F00089B200F092B8D05889B200F08CB8704718
:1026000000B9FEE703798B420FD901EB4101026863
:10261000CB00D118087D496818B1D05889B200F0B4
:102620007AB8D05889B200F078B87047FEE708B59C
:10263000FFF7FCFF08B5FFF7F9FF08B5FFF7F6FF56
:1026400008B5FFF7F3FF08B5FFF7F0FF08B5FFF790
:10265000EDFF08B5FFF7EAFF08B5FFF7E7FF08B59C
:10266000FFF7E4FF01BEFEE710B50446FEF7CEFB20
:10267000012806D11CB1FEF7C9FB013CF8E7052093
:1026800010BD002C08BF052010BDF0B500230E685A
:102690001C460125A54005EA060EAE452BD10F7953
:1026A0007A1E012A15D8856803229A4025EA02027B
:1026B00082604D7982689D4015438560828892B220
:1026C00022EA0E0282808A798588A2402A4392B249
:1026D0008280032205689A40D24315400560056850
:1026E0009F402F430760C7681740CA7902FA03F575
:1026F00047EA0502C2600134102C03F10203C8D17D
:10270000F0BD4FF6FF730360022200230371427194
:102710008371C3717047816170470185704701F013
:102720000703C90800EB810010B59B00046A0F2164
:10273000994024EA01010162016A9A401143016251
:1027400010BD4FF4165303600C22002343608360D6
:10275000C360026143617047036811B143F0010334
:1027600001E023F001030360704743680AB1194395
:1027700001E023EA010141607047436811B143F46D
:10278000004301E023F4004343607047836811B1C4
:1027900043F0080301E023F008038360704710B59D
:1027A000C1F307240123C9B2022C03FA01F301D1BA
:1027B000043002E0032C08BF083012B10268134352
:1027C00002E0026822EA0303036010BD836823F479
:1027D00080538360836819438160704710B5B2FBF2
:1027E000F0F4B4FBF1F301FB13434343B3FBF1F308
:1027F0004143B2FBF1F1C90748BFC31A00FB1424DF
:102800009C424FF0000003D9BDE81040FEF7A0BF86
:10281000BDE81040FEF7A4BF08B5FFF796FEBDE87F
:102820000840FFF7A2BE10B50020FDF70FFE0446DA
:102830000120FDF70BFE41F222139C4205D14AF61E
:102840005523C31A5842584110BD002010BD08B589
:1028500000200146FDF708FE01200021BDE80840E8
:10286000FDF702BE01460220FDF7FEBD4378027867
:102870001B0403EB0263C2788078134403EB00204F
:102880007047F8B505460F4662B9061D0446781B29
:102890002044FFF784FE037804F8013BB442F6D1EC
:1028A0000120F8BD0020F8BD00000000010000007C
:1028B000020000000300000004000000050000000A
:1028C00006000000070000000800000009000000EA
:1028D0000A0000000B0000000C0000000D000000CA
:1028E0000E0000000F00000045090008D508000890
:1028F000000000003507000815070008B1080008AF
:102900008D0800080000000000000000000000002A
:1029100000000000690900083C030020FF000000DF
:1029200040040020FF000100881300005D1400082F
:1029300015140008F91300083105000800040048C8
:10294000080000000103000000000000000000007B
:1029500000000000000800480080000001030000A3
:102960000000000000000000000000003C290008FA
:10297000020000000038014007000000000000488D
:1029800000040000020300010A00000000000048EB
:102990000002000002030001090000000000000026
:1029A0000000000000000000000000000000000027
:1029B00000440040070000000000004800800000C4
:1029C000020300010F00000000000048004000006A
:1029D000020300010E0000000000000000000000E3
:1029E000000000000000000000000000004800405F
:1029F0000700000000040048000800000203000176
:102A00000B00000000040048000400000203000165
:102A10000A000000000000000000000000000000AC
:102A200000000000000000000000C1C081C14001A2
:102A300001C3C003800241C201C6C006800741C76E
:102A40000005C1C581C4400401CCC00C800D41CD3E
:102A5000000FC1CF81CE400E000AC1CA81CB400B0E
:102A600001C9C009800841C801D8C018801941D9DE
:102A7000001BC1DB81DA401A001EC1DE81DF401F6E
:102A800001DDC01D801C41DC0014C1D481D540157E
:102A900001D7C017801641D601D2C012801341D38E
:102AA0000011C1D181D0401001F0C030803141F11E
:102AB0000033C1F381F240320036C1F681F740376E
:102AC00001F5C035803441F4003CC1FC81FD403D3E
:102AD00001FFC03F803E41FE01FAC03A803B41FB0E
:102AE0000039C1F981F840380028C1E881E940295E
:102AF00001EBC02B802A41EA01EEC02E802F41EF6E
:102B0000002DC1ED81EC402C01E4C024802541E57D
:102B10000027C1E781E640260022C1E281E340238D
:102B200001E1C021802041E001A0C060806141A19D
:102B30000063C1A381A240620066C1A681A740676D
:102B400001A5C065806441A4006CC1AC81AD406D3D
:102B500001AFC06F806E41AE01AAC06A806B41AB0D
:102B60000069C1A981A840680078C1B881B94079DD
:102B700001BBC07B807A41BA01BEC07E807F41BF6D
:102B8000007DC1BD81BC407C01B4C074807541B57D
:102B90000077C1B781B640760072C1B281B340738D
:102BA00001B1C071807041B00050C190819140511D
:102BB0000193C053805241920196C056805741976D
:102BC0000055C19581944054019CC05C805D419D3D
:102BD000005FC19F819E405E005AC19A819B405B0D
:102BE0000199C059805841980188C048804941895D
:102BF000004BC18B818A404A004EC18E818F404F6D
:102C0000018DC04D804C418C0044C184818540457C
:102C10000187C047804641860182C042804341838C
:0E2C20000041C1818180404004000500060093
:102C300000A24A0488130000640000006400000041
:102C400088130000010002000400060008000A00CA
:102C50000C00100020004000800000010000000077
:102C6000000000000000000000000000010203045A
:102C70000607080900000000010203040102030422
:082C800006070809010000002D
:103F8000BDBDBDBD10010001004000089CBF030085
:103F90009CFF030864000000000000000000000017
:103FA0000000000000000000000000000000000011
:103FB0000000000000000000000000000000000001
:103FC00000000000000000000000000000000000F1
:103FD00000000000000000000000000000000000E1
:103FE00000000000000000000000000000000000D1
:103FF00000000000000000000000000000000000C1
:0400000508000000EF
:00000001FF
